:100000000EC013C012C011C010C00FC00EC00DC072
:100010000CC00BC00AC009C008C007C006C011242C
:100020001FBECFEDCDBFD8D0EAC0EACF1ABC13BEF9
:10003000C398089583E28ABD89E083BF0895F89448
:1000400081E088BB82E087BB89E189BD8CE088BD07
:10005000789408951F93DF93CF930F92CDB7DEB7B7
:1000600018E08983E7DF90E99A95F1F7DFDF89816E
:1000700087FF07C0E4E4F1E03197F1F700C000002A
:1000800003C0F0E9FA95F1F7115011F0880FE9CFAC
:100090000F90CF91DF911F9108951F93DF93CF931E
:1000A00000D0CDB7DEB7182F6A837983C3DF81E52F
:1000B00093E00197F1F700C00000B8DFE7EBF1E053
:1000C0003197F1F700C0000080E4C4DF84E0C2DFB4
:1000D00085E0C0DF812FBEDF7981872FBBDF6A819A
:1000E000862FB8DFA7DFF0E9FA95F1F79FDF80EC04
:1000F00098E40197F1F700C00000CE5FCDBFCF912B
:10010000DF911F910895EF92FF920F931F937B0150
:100110008C01C3DFC801B701C0DFC801B701BDDF73
:100120001F910F91FF90EF9008950DC0E9EFF0E05F
:100130003197F1F700C000002F5F3F4FF1E0243FFF
:100140003F071CF0089520E030E0B09B02C08823F8
:1001500069F7B099F8CF882349F3F5CF8FE39DE095
:10016000A3E081509040A040E1F700C000008FE381
:100170009DE0A3E081509040A040E1F700C0000066
:100180008FE39DE0A3E081509040A040E1F700C0E4
:10019000000008951F9310E261E074E080E090E0B9
:1001A000B2DF8BE792E90197F1F700C00000115030
:1001B00099F71F9108951F9316E161E874E880E0B4
:1001C00090E0A1DF8BE792E90197F1F700C0000012
:1001D000115099F71F91089532DF80E0A6DF6CE59A
:1001E00079E580E090E08FDFB9DFD4DF81E09DDF4B
:1001F000E2DF61E87CEB88E390E085DFEECFF89406
:02020000FFCF2E
:00000001FF
